:020000040800F2
:10000000D80C0020D5000008AD190008690C0008C4
:1000100000000000000000000000000000000000E0
:10002000000000000000000000000000BB1E0008EF
:100030000000000000000000A91A0008E91F0008E5
:10004000E7000008E7000008E7000008E7000008F4
:10005000E7000008E7000008E7000008E7000008E4
:10006000E7000008E7000008E7000008E7000008D4
:10007000E7000008E7000008E7000008E7000008C4
:10008000E7000008E7000008E7000008E7000008B4
:10009000E7000008FD2000081D210008E700000817
:1000A000E7000008E7000008E70000085D210008FD
:1000B000A5210008ED210008E70000080448854656
:1000C00000F0E2FA004800473D2B0008C046C04659
:1000D000D80C00200448804704480047FEE7FEE7AC
:1000E000FEE7FEE7FEE7FEE7A1200008BD000008EE
:1000F00030B50B46014600202022012409E00D46C0
:10010000D5409D4205D31D469540491B2546954047
:1001100040191546521E002DF1DC30BD70B500248B
:100120002546002801DA01244042002901DA012590
:100130004942FFF7DDFFAC4200D04042002C00D026
:10014000494270BD10B5202A04DB0846203AD04051
:10015000002110BD0B46D340D0402024A21A91406C
:100160000843194610BDD2B201E00270401C491E7E
:10017000FBD270470022F6E710B513460A46044644
:100180001946FFF7F0FF204610BD421C0178401CC5
:100190000029FBD1801A704730B505460020034680
:1001A00000E05B1C934205D2EC5CC85C201A01D1D4
:1001B000002CF6D130BDF8B502464A40D40F4200BB
:1001C0004B0052085B089A4202D20246084611468A
:1001D0004A0023D0C30D4A00DDB2120EAD1A202D05
:1001E00035DA49020126490AF6058A19002C00D0A1
:1001F000524220214F1B1146B9402A411018C20D0E
:100200009A4221D0002C17D0012D08DCDA05801A83
:10021000D20F8019D207DBB200F09DF9F8BDDA05E4
:10022000801A012340001B06C01880185A4280180B
:10023000CA0F1043490007E04908C2071143DA0515
:10024000801A80194008801800F07DF9F8BD61001F
:100250000122511A001BF7E70122D2075140AAE7F9
:100260000122D2075040A6E7024670B54A40D30F9C
:10027000DB0740002DD04A002AD0010E140E0002E8
:1002800012020919400A520A8418E501044654432F
:10029000000A120A2E045043A4194219200CC54327
:1002A000AA18120C0125AD03521C521912047F39F1
:1002B000240400D0521C104301D44000491EC2B295
:1002C0000C06C0092018401C4008802A02D003E018
:1002D000002070BD40084000002900DA00201843CB
:1002E00070BD70B502464A40D50F40004A00ED0788
:1002F00040085208002814D0002A12D0C40DD30D93
:1003000041020120C0055202490A520AE41A0918A2
:1003100012187D34914201D3641C00E04900002C86
:1003200001DA002070BD0023914201D3891A0343F2
:10033000400849000028F7D100290AD0914202D193
:100340000121C90705E0914201D2012101E001210B
:10035000C943E005C018401900F0F5F870BD000071
:10036000F0B50C465C4085B0E40FE40703944C0004
:100370000026640859009446490802460296224322
:1003800021D062460A431ED06200570D4A000E0378
:100390002303550D012402462C492405781B1B0B11
:1003A000360B401823432643614600901C46501AE2
:1003B000B44103D30098401C009002E092180098CA
:1003C0005B41002803DA0020014605B0F0BD0020A3
:1003D000012109050746864611E064461D46141BA7
:1003E000B54106D36546521BB341744607430C43DF
:1003F000A646CD0740084908284392185B410546A8
:100400000D43EAD11046184313D0604619465040B8
:100410007140084306D06046101AB34106D201224B
:10042000002306E000220123DB0702E00122D24381
:100430005310009874460105381C6141029C039DCD
:100440000019694100F0C0F8BFE70000FD0300009B
:1004500010B500229623114600F07DF810BD000073
:100460000EB505490291002100910A460B46019103
:1004700000F0B7F803B000BD33040000C20F410024
:1004800040020123400ADB05D207090EC0187F296C
:1004900001DA00207047962903DC9623591AC840D8
:1004A00001E096398840002AF4D040427047CB0FD3
:1004B000DB07490010B5490802460A4307D00A0D78
:1004C00007240903E401090B121B002A01DC0020A8
:1004D00010BDC900440F0C43C100E018D2058018BC
:1004E00000F031F810BDF0B51FB40646002082B010
:1004F00005464024019100901BE0019922460F46D9
:100500003046FFF71FFE049A059B801A994110D3CD
:1005100010461946224600F0C9F8361A8F41019755
:10052000224601200021009F00F0C0F838184D41FC
:1005300000902046641E0028DFDC019B00982946BD
:10054000324607B0F0BD002904DA401C490001D151
:1005500040084000704770B40024050C05D11024F9
:10056000000402D1002921D01124050E01D100027E
:100570000834050F01D10001241D850F01D1800031
:10058000A41C002801DB4000641C002908D02025A1
:100590002E1B0D46F540A14000D001212943084300
:1005A00001061B1B000ADB1D02D5002070BC704732
:1005B000DB05181880180029F8DA401C4900F5D12D
:1005C00070BC40084000704710B5002B08DA0024CA
:1005D000401C614192185B411A4301D14008400020
:1005E00010BDF0B51FB482B005460C0003D008461C
:1005F00001F010FF02E001F00DFF203002460090F4
:100600002146284600F052F8049B059A04460F46FE
:1006100018431143084314D0184610431BD00098C8
:1006200040210A1A18460599FFF78CFD05460E462B
:10063000009A0599049800F039F8084305D0012084
:1006400004E02046394607B0F0BD0020C11705433D
:100650000E432C43374300990E986305401A7905E1
:10066000E40A00220C43FD0A0A3002D500200146AC
:10067000E9E70105101969410C9C0D9D00196941BC
:10068000FFF7A2FFDFE70000064C0125064E05E05C
:10069000E36807CC2B430C3C98471034B442F7D3A3
:1006A000FFF710FD1C2F00083C2F000810B5202A72
:1006B00004DB0146203A9140002010BD91402023E8
:1006C0009C1A0346E3401943904010BD10B50178D1
:1006D0000B0001F0B6FE050404070404060002F056
:1006E00033F910BD02F01CFB10BD1AE000BF00BFC3
:1006F00000BF00BF00BF00BF00BF00BF00BF00BF02
:1007000000BF00BF00BF00BF00BF00BF00BF00BFF1
:1007100000BF00BF00BF00BF00BF00BF00BF00BFE1
:10072000401E0028E2D170477047000006490020B3
:10073000C861064801690422114301610169402230
:100740001143016170470000B808002000200240FA
:10075000064A0021D16106490A6902231A430A6147
:10076000486108694022104308617047B8080020BA
:100770000020024010B5054B0022DA61044A1369DB
:10078000012423431361018010BD0000B80800203C
:100790000020024010B50B4A0020D168CB060A4960
:1007A00004D5C86902231843C8611020D3685B07C9
:1007B00005D5CB6901242343CB6104210843D060D4
:1007C00010BD000000200240B808002070B50546AA
:1007D00000F0E4F90646104C0AE0681C08D0002D31
:1007E00004D000F0DBF9801BA84201D9032070BDC2
:1007F000E068C007F1D1E068800601D52020E06004
:10080000E068C00602D4E068400703D5FFF7C2FFE6
:10081000012070BD002070BD00200240F8B53220DC
:1008200000F030FD07223F493F4801F0B9FD32207A
:1008300000F028FD3B4909220E313C4801F0B0FD93
:10084000322000F01FFD374909223231384801F0CB
:10085000A7FD322000F016FD32490922203135482B
:1008600001F09EFD322000F00DFD2E4909222031BD
:10087000314801F095FD322000F004FD2F4D32206B
:10088000009001230022291D284601F00DFAFF20C7
:100890002C462F68C00501262034C74201D226719C
:1008A00001E0002020713846FFF7E8FD607124491F
:1008B0003846FFF7D9FCFFF7E1FD6421FFF72EFC76
:1008C000A1716F683846FFF7D9FDE0711C493846C1
:1008D000FFF7CAFCFFF7D2FD6421FFF71FFC0127D9
:1008E0002172BF023946174800F076FB6074394622
:1008F000144800F071FBC0B2A074617C002908D0DC
:10090000012905D100280AD0012801D10320A861BE
:10091000F8BD0028FBD00128FAD1AE61F8BD022055
:10092000F5E70000302E0008004C004000140140A4
:100930000048004000500040003801407C08002082
:100940000000C8420004004800B50179002907D022
:10095000C268816800F010F8002809D0012000BDAD
:1009600002680449516100688168182291438160DE
:10097000002000BDB71DC10430B51F2301252C4642
:100980009C400C4201D15B1EF9D2002A0FD0082AEC
:1009900009D0102A04D0182A09D1072B05D206E065
:1009A000082B02D203E0102B01D3012030BD0368D5
:1009B00059610168886818239843104388600020B3
:1009C00030BD10B504000DD0607F002803D1207722
:1009D000204600F025F8022060772046FFF7B4FF9C
:1009E000002801D0012010BD6079002814D02069B2
:1009F0002168086121688868602290436269104319
:100A000088602168886880229043A26910438860CA
:100A100001206077002010BD0020C043E8E70000FF
:100A200008B500680549884207D105484269402158
:100A30000A43426140690840009008BD003002400E
:100A400000100240F8B5054623480F46017E0126F6
:100A500001290BD0012101762868204C012807D0FC
:100A60002046FFF7B3FE002813D030E00220F8BD87
:100A70002046FFF7ABFE002829D1FFF757FE20469E
:100A8000FFF7A4FE0646164801690422914301615E
:100A90001DE00020C04338606C6812E02046FFF77C
:100AA00057FE0E48FFF792FE06460D4802690221E6
:100AB0008A430261002E01D03C6008E00120C002A0
:100AC0002418A868C10268680818A042E6D802483D
:100AD000002101763046F8BDB808002050C3000060
:100AE0000020024003480169802211430161002077
:100AF0007047000000200240F0B51FB407461A48B6
:100B00000024017E15461E46012907D001210176E9
:100B10001648FFF75BFE002803D020E0022005B056
:100B2000F0BD012F02D0022F00D004272201284659
:100B30003146FFF707FB81B2019862001018FFF7FA
:100B400019FE0A48FFF742FE09490A695208520095
:100B50000A61002803D1641CE4B2BC42E6D3024916
:100B600000220A76DBE70000B808002050C300002E
:100B700000200240064900200A69120607D5054AEE
:100B80004A60054A4A600969090600D50120704794
:100B90000020024023016745AB89EFCD0148006882
:100BA000704700003400002002480168491C0160C1
:100BB000704700003400002010B50648016810227C
:100BC00011430160002000F007F800F017F8002042
:100BD00010BD00000020024010B5044600F026F8C9
:100BE0007D21C900FFF784FA00F026F80022214693
:100BF000501E00F017F8002010BD000008B508488E
:100C00008169012211438161816911400091C269AA
:100C100001040A43C261C0690840009008BD000099
:100C20000010024010B500F011FF10BD014800682F
:100C30007047000030000020094910B5401E88426E
:100C400001D9012010BD074C60610321081F00F08D
:100C5000FDFE0020A06107202061002010BD0000E3
:100C6000FFFFFF0000E000E0FEE7000000B50D48D8
:100C700087B0816908221143816101150920C006EE
:100C80008161491081610321490200910121019193
:100C900003910321029100210491694600F048F973
:100CA00007B000BD00100240F7B5009800210170A8
:100CB000012080020924E406A06180260120400270
:100CC000A0610120FFF711FD0027029D08E02846E2
:100CD0006D1EEDB2002832D07D20C000FFF705FD6B
:100CE00020698005F3D50320FFF7FFFC206940054C
:100CF00004D5009800990078304308700120400620
:100D0000A0610120FFF7F1FC7608D7D101980028F7
:100D100017D001208002A0610120FFF7E6FC01202E
:100D20004002A0610520FFF7E0FC01204006A06121
:100D3000C013A0611420FFF7D8FC3846FEBD04277D
:100D4000D1E701208006E6E710B5012080020924E2
:100D5000E406A0610120FFF7C8FC01204002A06169
:100D60000120FFF7C2FC01208006A0610A20FFF7E6
:100D7000BCFC01204006A0610A20FFF7B6FC10BDB4
:100D800010B5012040060924E406A0610120FFF708
:100D9000ACFC01208006A0610120FFF7A6FC012029
:100DA0004002A0610A20FFF7A0FC01208002A061A0
:100DB0000A20FFF79AFC10BDF1B58025002082B013
:100DC000AE00AF040924E40600900298054202D167
:100DD0000120800601E001208002A0610120FFF7D0
:100DE00084FCA6610520FFF780FCA7610120FFF7C6
:100DF0007CFC6D08E9D101208002A061A661012080
:100E0000FFF773FC2069400501D501200090A76120
:100E10001420FFF76AFC0098FEBD10B5801C00F09E
:100E200002FF10BD70B5044602700D46801C00F034
:100E3000FAFEFF20493005550020FF340134E064FC
:100E400070BD000019490160194941607F21C90541
:100E500081601849C1600161FF2191314161002128
:100E600081611421C1611921016220304171372152
:100E700081712B21C1712E21017205224272042140
:100E800081720723C3721223037341734E2383734A
:100E9000C173702101740121417481740221C174F4
:100EA0002D21017542758175704700000000D04109
:100EB000000048420AD7233C08B504494A69024366
:100EC0004A6149690140009108BD000000100240DC
:100ED00008B504494A6902434A61496901400091E1
:100EE00008BD00000010024008B50449CA69024369
:100EF000CA61C9690140009108BD000000100240AC
:100F000008B504498A6902438A61896901400091F0
:100F100008BD00000010024008B504498A69024378
:100F20008A6189690140009108BD000000100240FB
:100F3000F0B500243EE001232A46A3401A4038D0F1
:100F40004F680668134653435D005D19AE435F4327
:100F50003E4306604E68012E01D0022E05D18F68F7
:100F600086685F43AE433E4386600F69C668AE4302
:100F70001D467D432E43C6604D68022D19D1FF2AC0
:100F80000AD84E69056A534353431A01D21A95434E
:100F900073431D4305620CE0130A1A465A435A4331
:100FA0005A4313019E1A4D69436A6A43B34313437C
:100FB0004362641C0A681546E240BCD14A68012AB3
:100FC00001D0022A06D1CB6841682A4691435A4390
:100FD000114341600120F0BD0069814301D0002030
:100FE00070470120704710B5044600F079FD20607D
:100FF00000F05CFD606000F067FDA06010BD0000C7
:1010000070B5012600241F4DF603002804D01028D7
:101010000BD0122820D01DE000F03AF801282DD086
:10102000022812D0032822D109E000F031F8164935
:10103000411823D00120000415E004460AE000F026
:1010400031F8002806D02C4604E000F033F80028E0
:1010500000D03446204670BD00F01AF80B49411804
:101060000CD001208004091AEFD08142E7D000F0B3
:1010700037FD00F01BFD00F027FDDEE700F030FD3E
:10108000DBE7000000127A000000FFEF0000FCED3B
:101090000349096B03228240114000060843704750
:1010A00000100240024800688007C00F704700002F
:1010B000001002400248006A8007C00F704700001D
:1010C0000010024010B505490A6B040E0323A3402B
:1010D00000029A43000A02430A6310BD0010024056
:1010E000014908607047000030000020F0B5026838
:1010F0001D4B0124A4071D4D984203D0A04201D0EE
:10110000A84203D17026B2434E683243184E194F9D
:1011100098420DD0A0420BD0A84209D0164CA04254
:1011200006D0B04204D0B84202D0144CA04204D140
:1011300003242402A243CC68224302608A68C2626C
:101140000A888262984206D0B04204D0B84202D0E7
:101150000A4A904201D1097C01634169012211438D
:1011600041611046F0BD0000002C01400004004029
:101170000040014000440140002000400048014080
:1011800041680922D2029143416081682A22914339
:1011900081607047FEB5044600680D460026C00712
:1011A000C00F59D1E9686868AA69084329691143E1
:1011B00008432168294A114008432060A9686068F3
:1011C000032212039043084360606969A06812110A
:1011D00090430843A0602248844201D1002008E0E7
:1011E0002048844201D1102003E01F48844203D1EB
:1011F0001220FFF705FF12E01C4884420BD01C4868
:10120000844208D01B48844205D01B48844202D047
:101210001A48844220D16846FFF7E5FE029800286C
:101220001AD02968002917D00126AA69F3039A4227
:101230000CD140004A088018FEF75AFF81B21048CE
:1012400008400907490F0143E16005E04A0810180A
:10125000FEF74EFF80B2E0603046FEBDF369FFEF5F
:10126000003801400044004000480040004C00406D
:10127000005000400014014000180140001C0140D3
:10128000F0FF000008B506490A690092421C00D030
:10129000401C0A69D20300D5401E0028F9D108BDC0
:1012A00000E000E010B50948074901600021017124
:1012B00041714161816101210162FFF782FB0028D8
:1012C00001D0FFF731FA10BD003002403800002095
:1012D000F0B587B018216846FEF74CFF0120800565
:1012E000FFF7EAFD0120C004FFF7E6FD01204004FE
:1012F000FFF7E2FD01208004FFF7DEFD012000057D
:10130000FFF7DAFD274E0420B0610820B0614701E5
:101310000920C00687612449F8018862002404205E
:101320000125009002940394694601950494304687
:10133000FFF7FEFD08200090029403946946019592
:1013400004943046FFF7F4FD019469461648009571
:101350000494FFF7EDFDA8020090019469460494FF
:101360001148FFF7E5FDE8020090019469460494F6
:101370000D48FFF7DDFDE8030090029403946946F1
:10138000019504940848FFF7D3FD092002940394C3
:101390006946C006009701950494FFF7C9FD07B0A0
:1013A000F0BD000000080048000400480849074854
:1013B0000860084808600320486007488860CA68D9
:1013C0005207FCD10861054808607047CCCC00008A
:1013D0000030004055550000FF0F0000AAAA000091
:1013E00010B586B014216846FEF7C4FE0120400403
:1013F000FFF786FD0021152000F0E4FA01200B49DB
:10140000400508600A4869460880002009490291A1
:10141000019003906946084C08742046FFF766FE69
:10142000206880218843206006B010BD00E100E004
:1014300080BB0000B80B00000044014010B586B02E
:1014400014216846FEF796FE01208004FFF758FD40
:101450000021162000F0B6FA01200B498005086033
:101460000A486946088000200949029101900390CA
:101470006946084C08742046FFF738FE2068802132
:101480008843206006B010BD00E100E07FBB000093
:101490008713000000480140F0B58DB01C2106A85C
:1014A000FEF768FE18216846FEF764FE01208003FF
:1014B000FFF732FD01208004FFF70AFD00244020E1
:1014C00002250326039404946A46059461C2194FC9
:1014D00069463846FFF72CFD8020039404946A4641
:1014E000059461C269463846FFF722FD01211B20A1
:1014F00000F08AFA1B2000F05BFA4B20C001069036
:101500000794089409940B940C940C200A4C0A90AC
:1015100006A92046FFF73EFEA06821158843A0607B
:101520002046FFF72DFE20680121084320600DB002
:10153000F0BD00000004004800380140F0B58DB057
:101540001C2106A8FEF716FE18216846FEF712FEBB
:10155000012464042046FFF7C7FC2046FFF7B8FCCF
:101560000024012504200226032703946A460595DA
:101570000494C1C209206946C006FFF7D9FC0820BF
:1015800003946A4605950494C1C209206946C006C1
:10159000FFF7CEFC01211C2000F036FA1C2000F0E1
:1015A00007FA4B20C00106900794089409940B9405
:1015B0000C940C20084C0A9006A92046FFF7EAFD7F
:1015C000A06821158843A0602046FFF7D9FD206858
:1015D000284320600DB0F0BD00440040F0B58DB050
:1015E0001C2106A8FEF7C6FD18216846FEF7C2FDBD
:1015F00001208004FFF778FC0120C004FFF768FC9D
:101600000024012510200226032703946A4605952D
:101610000494C1C269461748FFF78AFC202003944E
:101620006A4605950494C1C269461248FFF780FCDA
:1016300001211D2000F0E8F91D2000F0B9F94B2030
:10164000C00106900794089409940B940C940C2004
:10165000094C0A9006A92046FFF79CFDA0682115B9
:101660008843A0602046FFF78BFD20682843206058
:101670000DB0F0BD0008004800480040F0B58DB046
:101680001C2106A8FEF776FD18216846FEF772FDBC
:101690000120C004FFF728FC01204004FFF718FCDC
:1016A0000126042000960024059002250327092026
:1016B00003946946029701950494C006FFF738FC2D
:1016C000009504200590092003946946029701952E
:1016D0000494C006FFF72CFC01211D2000F094F9B2
:1016E0001D2000F065F94B20C00106900794089476
:1016F00009940B940C940C20084C0A9006A92046DF
:10170000FFF748FDA06821158843A0602046FFF739
:1017100037FD2068304320600DB0F0BD004C004024
:1017200070B58EB01C2106A8FEF724FD182168466E
:10173000FEF720FD012424052046FFF7D5FB6010AD
:10174000FFF7C6FB2046FFF7C3FB2012002402254B
:10175000032603946946049461C1694618480595B7
:10176000FFF7E6FB042003946946049461C16946CF
:1017700014480595FFF7DCFB01211D2000F044F91A
:101780001D2000F015F94B20C00106900794089425
:1017900009940B940C940C200B4C0A9006A920463B
:1017A000FFF7F8FCA06821158843A0602046FFF7EA
:1017B000E7FC20680121084320600EB070BD0000E6
:1017C00000080048000C004800500040F0B58DB003
:1017D0001C2106A8FEF7CEFC18216846FEF7CAFCBD
:1017E0002020FFF799FB01204004FFF771FB002444
:1017F000052710200225032603946A4605970494C2
:1018000061C209206946C006FFF792FB20200394BD
:101810006A460597049461C209206946C006FFF72D
:1018200087FB01211D2000F0EFF81D2000F0C0F81B
:101830004B20C00106900794089409940B940C94D3
:101840000C20094C0A9006A92046FFF7A3FCA068CB
:1018500021158843A0602046FFF792FC20680121F3
:10186000084320600DB0F0BD00140140F0B58DB00C
:101870001C2106A8FEF77EFC18216846FEF77AFCBC
:101880004020FFF749FB0120C004FFF721FB0024A3
:10189000012540200226032703946A4605950494F7
:1018A000C1C269461748FFF743FB802003946A468C
:1018B00005950494C1C269461248FFF739FB01211E
:1018C0001D2000F0A1F81D2000F072F8E120400278
:1018D00006900794089409940B940C940C200A4CDD
:1018E0000A9006A92046FFF755FCA06821158843F9
:1018F000A0602046FFF744FC2068284320600DB01C
:10190000F0BD00000008004800180140F0B58DB09F
:101910001C2106A8FEF72EFC18216846FEF72AFCBB
:101920008020FFF7F9FA0120C004FFF7D1FA002464
:10193000FF20012501300226032703946A460595FE
:101940000494C1C269461748FFF7F2FA680203948B
:101950006A4605950494C1C269461248FFF7E8FA41
:1019600001211D2000F050F81D2000F021F84B202F
:10197000C00106900794089409940B940C940C20D1
:10198000094C0A9006A92046FFF704FCA06821151F
:101990008843A0602046FFF7F3FB206828432060BF
:1019A0000DB0F0BD00080048001C01407047000069
:1019B000C106C90E01208840014908607047000037
:1019C00000E100E08307FF22DB0E9A408907090E41
:1019D000994000280BDA0007000F083883080848F0
:1019E0009B001818C36993430B43C3617047830876
:1019F00004489B001B181868904308431860704700
:101A000000ED00E000E400E08307FF22DB0E9A40D7
:101A10008907090E994000280BDA0007000F0838E3
:101A2000830808489B001818C36993430B43C3619C
:101A30007047830804489B001B18186890430843AC
:101A40001860704700ED00E000E400E08307FF222B
:101A5000DB0E9A408907090E994000280BDA00072F
:101A6000000F0838830808489B001818C36993437F
:101A70000B43C3617047830804489B001B18186818
:101A8000904308431860704700ED00E000E400E078
:101A900010B510220249034800F082FC10BD00007E
:101AA000202E0008001C01407047000004494968CE
:101AB000F0221140034A0909515CC84070470000F8
:101AC00000100240742E000803494968034A490582
:101AD000490F515CC840704700100240842E000836
:101AE00010B5094841680C200140084806D0042977
:101AF00005D0082905D00C2900D1054810BD05489E
:101B000010BD00F009F810BD0010024000127A006C
:101B1000006CDC020024F40010B50F4C6068032157
:101B2000C90308400121C903421A0C4806D0521AC1
:101B300003D08A4202D10A4800E00A48E16A090754
:101B4000090F491CFEF7D4FA61680F229204114074
:101B5000890C891C484310BD0010024000127A0015
:101B6000006CDC020024F400F8B5064600240C4D9D
:101B70000EE0684601782819FF300130641C0172BC
:101B8000802C05D36946304600F039F80028F9D199
:101B90006946304600F033F80028EAD1F8BD00006D
:101BA0005C000020F8B504460025801C00F025F8F4
:101BB0002646FF3601464136307A814216D26946C2
:101BC000A01C00F01CF80028F9D1F8BD6846017887
:101BD0006019FF3001300172307A6D1CA84205D8BF
:101BE0006946A01C00F00BF80028F9D16946A01C3A
:101BF00000F005F80028E9D1F8BD00797047828827
:101C0000002A0ED002885200121892790A700178C8
:101C1000491C4906490E01808188491E81800120A6
:101C2000704700207047002101804180818070470B
:101C300070B50546FF200022FF2432340FE0AB5C74
:101C400058400823060602D54000604000E04000EE
:101C50005B1E1B06C0B21B0EF4D1521CD2B28A42CC
:101C6000EDD370BD10B5FEF7F3FB0349FEF7FCFAA8
:101C70000249FEF736FB10BD0000C84200FF7F4757
:101C800010B5FEF7E5FB0549FEF7EEFA0449FEF74D
:101C900028FB0449FEF7E0FA10BD000000002F43C6
:101CA00000FF7F470000344210B5029C002B03D098
:101CB000012B05D0802010BD234600F005F810BD93
:101CC000234600F043F810BDFFB583B015460E461D
:101CD000074600F0DBF8040025D1002D0CD0012DC3
:101CE00007D0022D03D08024FFF74AF829E01648D8
:101CF00004E01548C01E01E013480A3800F0D0F88F
:101D0000040010D100F0B8F804000CD1002168469E
:101D1000069A00F080F8040005D10022012101A8F4
:101D200000F079F80446FFF72BF8002C09D168463B
:101D30000088FFF7A5FF386068468088FFF792FFAC
:101D40003060204607B0F0BD102C0000FFB583B016
:101D50001D461746064600F099F8040038D1002FBA
:101D60000AD0012F05D0022F01D0802430E0214875
:101D700004E020480B3801E00920800200F090F8D0
:101D8000040008D024E000F077F804000AD03846B8
:101D9000FEF7ABFC01E07D27FF0028466D1EEDB28B
:101DA0000028F0D1002D02D0002C04D010E0042433
:101DB000FEF7E6FF1BE000221146684600F02BF814
:101DC00005460022012101A800F025F804462C4315
:101DD000FEF7D6FF002C0AD168460088FFF750FFB7
:101DE000306068468088FFF73DFF04990860204610
:101DF00007B0F0BD1624000010B50446FEF736FF0C
:101E0000012080020921C9068861401088612046AE
:101E100000F028F810BD7CB50D4604460021684648
:101E2000FEF742FF002818D1002200A81146013019
:101E3000FEF73AFF002810D10022294601A8FEF73C
:101E400033FF002809D1684602210579FFF7F0FE2B
:101E5000A84201D0022000E000206946098849BA62
:101E600021807CBD03494000087001221043487066
:101E7000704700000900002010B5FEF765FF02481A
:101E80004078FEF799FF10BD0900002010B5FEF75D
:101E90005BFF02480078FEF78FFF10BD09000020AD
:101EA00070B50446000AFEF787FF0546E0B2FEF76C
:101EB00083FF01462943084670BD704730B504468C
:101EC0001948A1B0007803282CD1402111A8FEF7B1
:101ED00051F9214620318D7D4B7D0A7DC87C0D90C6
:101EE0000EA82CC0A0690C7CCB7B8A7B0C9009A827
:101EF0001CC0887A4C7B0B7BCA7A05AD1DC58879DE
:101F00004C7A0B7ACA7901AD1DC5487900900B79DE
:101F1000064A402111A800F061FAC2B211A9044892
:101F200000F03EFA21B030BD08000020BC2E0008B1
:101F3000001C014010B53220FFF7A4F9072219490F
:101F4000194800F02DFA3220FFF79CF915490922B3
:101F50003431164800F024FA3220FFF793F9114982
:101F600009222231124800F01BFA3220FFF78AF9C9
:101F70000C49092222310F4800F012FA3220FFF7F3
:101F800081F90849092210310B4800F009FA322082
:101F9000FFF778F94420FFF72FFF3220FFF772F99F
:101FA00010BD0000372E0008004C004000480040E3
:101FB0000050004000380140001401400268012137
:101FC0000A430260CA1E0261C2680A43C2607047C7
:101FD00001684908490001600121C9430161C168E4
:101FE00049084900C160704710B5FEF7DDFD10BD1E
:101FF00010B52848012102688A430A43026000683C
:102000002548016801221204114301600168890317
:10201000C90FFBD0416A012211434162416A89071D
:10202000C90FFBD041687B22D203914305221204E1
:1020300011434160C16A09090901C16201680122B5
:1020400012061143016001688901C90FFBD0416884
:10205000F02291434160416807221202914341609E
:1020600042680221920892000A4342600C224168B1
:1020700011400829FBD10948FFF732F80020FFF78B
:1020800021F801200007FFF71DF809204006FFF79F
:1020900019F810BD0020024000100240006CDC0264
:1020A000124801680122114301604168104A114041
:1020B000416001680F4A11400160016801229204E9
:1020C0009143016041683F22120491434160C16A1B
:1020D00009090901C162016B074A11400163416BA3
:1020E00049084900416300218160704700100240A7
:1020F0000CB8FF08FFFFF6FEACFEF0FF05480169D3
:10210000C907C90F04D0044A01211170C91E016119
:1021100070470000004401400200002010B50C4C44
:102120002046FFF755FF00F03BFE0A490A4A0B68BC
:10213000984203D800200860022000E001201070BF
:102140000868401C08602046FFF738FF10BD0000FB
:1021500000480140040000200100002010B50E4C92
:10216000E0690007C00F01D008202062E069800606
:10217000C00F04D0A08CC1B2084800F01CF9E0697F
:10218000C006C00F06D01020206205480178012249
:102190001143017010BD000000380140EE01002025
:1021A0000000002010B50E4CE0690007C00F01D000
:1021B00008202062E0698006C00F04D0A08CC1B264
:1021C000084800F0F8F8E069C006C00F06D01020FB
:1021D00020620548017820221143017010BD0000E3
:1021E000004400405E00002000000020F8B53E4D95
:1021F000E86908270007C00F002800D02F62E869AF
:102200008006C00F04D0A88CC1B2384800F0D3F8C3
:10221000E8691026C006C00F354C002803D02E6296
:10222000207830432070334DE8690007C00F00D09C
:102230002F62E8698006C00F04D0A88CC1B22E4876
:1022400000F0B9F8E869C006C00F04D02E6220780B
:10225000042108432070294DE8690007C00F00D011
:102260002F62E8698006C00F04D0A88CC1B2244850
:1022700000F0A1F8E869C006C00F03D02E622078F4
:10228000384320701F4DE8690007C00F00D02F624F
:10229000E8698006C00F04D0A88CC1B21A4800F0CB
:1022A0008AF8E869C006C00F04D02E6220780221A7
:1022B00008432070154DE8690007C00F00D02F6259
:1022C000E8698006C00F04D0A88CC1B2104800F0A5
:1022D00072F8E869C006C00F04D02E622078202171
:1022E00008432070F8BD0000001401408E04002057
:1022F00000000020004C0040DE05002000480040A7
:102300002E070020005000403E030020001C01402A
:102310005E0000201C4A908C10201062136820215F
:102320000B431360136803431360184A938C1062C5
:1023300013680B431360136803431360144A938CB0
:10234000106213680B431360136803431360114A50
:10235000938C106213680B4313601368034313607C
:102360000D4A938C106213680B4313601368034388
:1023700013600A4A938C106213680B431360116850
:102380000143116070470000001C0140001401402F
:10239000004C004000480040003801400050004020
:1023A00006E00B780385491CC3691B06DB0FFBD0D5
:1023B000521EF6D270478288802A01D300207047CF
:1023C000428852001218D1808178491C4906490E72
:1023D00041808188491C8180012070470FB47CB501
:1023E0000C0009AD01D0611E00E0002101910090B8
:1023F000074B6A462946089800F040F8002C02D0A6
:10240000009A002111707CBC08BC04B01847000081
:10241000F12800082021020C01D010211046020AE8
:1024200001D010460839020901D01046091F820860
:1024300001D01046891E420801D0881E7047081A34
:10244000704730B47446641E2578641CAB4200D2D9
:102450001D46635D5B00E31830BC184702E008C806
:10246000121F08C1002AFAD170477047002001E00E
:1024700001C1121F002AFBD170470000FFB591B0C7
:102480000F460546002606E025280AD0149A13991F
:1024900090476D1C761C28780028F5D1304615B081
:1024A000F0BD002400940121F34A029400E00443AB
:1024B0006D1C2B780846203B98401042F7D12878B5
:1024C0002A280ED00222287801463039092915D849
:1024D00000990A2359433039401814436D1C009069
:1024E000F1E701CF0090002805DA01204003044302
:1024F000009840420090022004436D1C28782E284A
:1025000015D10420044368786D1C2A280AD101CF14
:102510006D1C02900BE002990A2251433039401899
:102520006D1C02902878014630390929F3D92878A2
:102530006C2810D006DC4C281AD068280ED06A28E7
:1025400017D104E0742813D07A2812D110E00120AA
:10255000400504430CE00121090501E003210905C0
:102560000C436978814203D10120000524186D1CB9
:102570006D1C28786E281ED00CDC632831D004DC5A
:1025800000288BD0582811D1B2E064287BD069286C
:102590000CD178E073282DD004DC6F2870D070281F
:1025A00004D1A7E075286CD078286BD0149A1399C1
:1025B0009047761C62E06002400F022807D0032893
:1025C0000AD0042838680AD006603F1D56E03868F3
:1025D000F11706604160F8E738680680F5E7067095
:1025E000F3E73878694608740020487404A803901B
:1025F000012003E0386803900020C0433F1D6107BD
:102600000FD5002101E00199491C029A01919142E4
:1026100013DA8142F7DB019A0399895C0029F2D130
:102620000BE0002101E00199491C01918142FADB94
:10263000019A0399895C0029F5D101990098139AB0
:10264000401A00902146149B00F03CF90199801932
:10265000461807E0039803990078491C0391149ADF
:10266000139990470198401E0190401CF2D12146D9
:10267000149B139A009800F015F986196D1C0AE74F
:1026800041E033E034E00A2000210490059160022B
:10269000410F022905D001CFC2179446032905D066
:1026A00007E0FF1DFF08FF0003CF06E000B2C217DE
:1026B0009446042902D140B2C1178C4600226146DB
:1026C000944506DA0A460021404291418C462D216C
:1026D00002E0210504D52B216A461176012103E091
:1026E000E10701D02021F7E7019155E00A200BE036
:1026F000102009E010200490002104200443082049
:102700000591029003E008200021059104906002E9
:10271000410F022905D001CF00229446032906D09B
:1027200006E0FF1DFF08FF0003CF8C4603E080B2E8
:10273000042900D1C0B20021019121072CD52978AC
:102740000391702906D0049A1021059B4A401A4330
:1027500005D00EE040216A461176012108E061466D
:10276000014306D030216A46117603995176022141
:102770000191049A0821059B4A401A430CD16146F5
:10278000014301D1610707D530216A461176012145
:1027900001910299491E02912978582904D037A144
:1027A00003910FA90F910DE039A1F9E76146059B4F
:1027B000049AFDF798FE039B8C469B5C0F9A521E71
:1027C0000F92137061460143F0D10F9807A9081AC0
:1027D00020300390600704D5012000048443029850
:1027E00001E0012002900399884201DD401A00E0D7
:1027F000002041180290019809180098401A009092
:10280000E00306D42146149B139A009800F05AF86E
:1028100086190020049008E006A9085C149A139910
:1028200090470498401C761C049001998842F3DB81
:10283000E0030CD52146149B139A009800F042F84F
:10284000861904E0149A302013999047761C029957
:10285000481E02900029F5DC08E00F980F990078D7
:10286000491C0F91149A13999047761C0399481E9E
:1028700003900029F1DCFAE60928010030313233F7
:1028800034353637383961626364656600000000AC
:102890003031323334353637383941424344454696
:1028A00000000000F8B5044600251E4617468804BF
:1028B00004D405E039462020B0476D1C641EF9D5CC
:1028C0002846F8BDFFB50446002581B01E46C80362
:1028D00001D5302700E02027880404D505E03846DC
:1028E0000399B0476D1C641EF9D5284605B0F0BDAC
:1028F0004A68002A06D00A68531C0B6010704868AA
:10290000401E48607047000070B586B0064614212E
:102910006846FDF72FFC0B4D00240096E000295877
:1029200008223046FDF738FC002804D0641C042C33
:10293000F4D306B070BDE10049194A6820466946E3
:102940009047F6E70C000020F8B50446FF30013050
:10295000017AFF297DD1417A86297AD1FF21493137
:10296000095D002301224D1E06E0A618FF36013640
:10297000367AF318DBB2521C9542F6DCDA43234672
:10298000FF330833521CC95CD2B291426AD1394E2E
:1029900021783546384F203500292AD0012944D0E6
:1029A00003290AD004295DD1817AC07A0902081866
:1029B00001127061E973287454E0817BC07B0902C5
:1029C0000818FDF74DFD00222C4BFDF7C9FCFDF763
:1029D0006EFD07463061FDF751FD687328493846A2
:1029E000FDF742FCFDF74AFD6421FDF797FBA97353
:1029F00038E0817AC07A09020818FDF731FD00221B
:102A00003B46FDF7ADFCFDF752FD0746B060FDF714
:102A100035FD68721A493846FDF726FCFDF72EFD94
:102A20006421FDF77BFBA9721CE0817AC07A090260
:102A30000818FDF715FD00223B46FDF791FCFDF758
:102A400036FD0746F060FDF719FDE8720C4938467F
:102A500000E00DE0FDF708FCFDF710FD6421FDF737
:102A60005DFB29732046FF3040210930FDF782FBD2
:102A7000F8BD00007C0800200000594000408F4055
:102A80000000C84270B50D46002404E02868005DCF
:102A90003C2806D0641C2868FDF777FBA042F5D8D7
:102AA00070BD2868A41C005D30380300FFF7C9FC26
:102AB0000907090D0F111315181B0600F0E7062072
:102AC00000E00C2000F07EF970BD2420FAE73C20E5
:102AD000F8E77820F6E7B420F4E7FF206930F1E763
:102AE0002D200001EEE7FF20ECE7000010B50C46BA
:102AF0000F49C0000858FDF748FB216803220C5C11
:102B00000C49303C0C482300FFF79BFC05040608E9
:102B10000D0D0C00002202E0012200E002220A70EA
:102B2000FFF756FA10BD0A70FFF748FA10BD000013
:102B30000C000020080000200048014008B5FEF706
:102B40003BF8FFF755FAFEF7C3FBFEF777FCFEF7FD
:102B5000F5FCFEF7A7FBFEF79FFCFEF73FFDFEF737
:102B60008DFDFEF7DDFDFEF731FEFEF77FFEFEF781
:102B7000CDFEFEF71BFCFEF733FC7D200001FEF7C7
:102B800081FB00F013F900F00BF97D24E400A04272
:102B900002D90C2000F016F92046FEF773FB5148CD
:102BA000FEF73BF95048FEF74DF9042209214F4842
:102BB000FEF738F9022220214D48FEF733F90322AF
:102BC00009214C48FEF72EF9002209214A48FEF758
:102BD00029F9012209214948FEF724F9FFF79AFB58
:102BE000FFF7A8F9464D474C474E484F60780028FC
:102BF0000FD06078012802D0022808D102E0FDF74A
:102C00000DFE04E0FEF744FF3748FFF757F90020B8
:102C100060702078C00709D02078400840002070FC
:102C20003548FEF7BFFF3448FDF750FD2078800798
:102C300009D52078FD21084020703048FEF7B2FF0A
:102C40002E48FDF743FD2078C00609D52078EF21F6
:102C5000084020702548FEF7A5FF2448FDF736FD03
:102C60002078000709D52078F721084020702148F6
:102C7000FEF798FF1F48FDF729FD2078400709D58A
:102C80002078FB21084020701948FEF78BFF184878
:102C9000FDF71CFD207880060FD52078DF21084045
:102CA00020701048801CFEF75FFF19480090FFF766
:102CB0002BFE80210098FDF75DFA287803280FD0BD
:102CC0001448FFF77BF9A078012809D11148FFF7D4
:102CD0007FF90020A0700D220F491048FFF760FB1C
:102CE0003E6083E75C0000207C0800208C0400200C
:102CF000DC0500202C070020EC0100203C03002014
:102D00000800002000000020AAAA000000300040B7
:102D10006401002000440140082E0008001C01400E
:102D200070B5C11DF9310A7A0023422A34D14A7A9A
:102D30004D2A31D1FF244934245C0022A41E06E030
:102D40008518FF3501352D7AEB189BB2521C944241
:102D5000F6DC0246FF32213295791C0AAC4216D1CC
:102D6000D279DBB2934212D10A7D4B7D12020B4C19
:102D7000D218E2618B7DC97D1B025B180749236273
:102D800014122031CC740A751A124A758B75FF30F3
:102D900040210930FDF7EEF970BD00007C080020ED
:102DA00001480068008870472C00002010B50B22F5
:102DB00002490348FFF7F4FA10BD0000152E000881
:102DC000001C014030B585B00446FDF7D3FE00205D
:102DD0000C4D00902968019101210291049004A9F1
:102DE0006846FDF72FFE002809D122460023012066
:102DF0002968FDF781FE0446FDF774FE204605B004
:102E000030BD00002C00002041542B535441545538
:102E1000533D3F0D0A41542B5245424F4F540D0A2A
:102E200041542B43555252454E5444523D350D0AA0
:102E3000424DE200000171424DE100000170FF01CE
:102E400086000000000079FF019900000007D08F84
:102E5000FF0186000000000079FF017804000000F7
:102E60000083FF0186000000000079FF0178410027
:102E70000000004600000000000000000102030402
:102E80000607080900000000010203040D0A2B5385
:102E900054415455533A00000D0A5E535441545561
:102EA000533A00005E5354415455533A0000000019
:102EB0000D0A5E4C52524543563A000041542B4C89
:102EC0005253454E443D3130312C302C31382C3C5E
:102ED00025303278253032782530327825303278F6
:102EE00025303278253032782530327825303278E6
:102EF00025303278253032782530327825303278D6
:102F000025303278253032782530327825303278C5
:102F100025303278253032780D0A00003C2F000829
:102F200000000020380000005C240008742F000816
:102F300038000020A00C00006C24000800000000F5
:102F400000000000020000008C2E0008ED2A00089E
:102F5000982E0008ED2A0008A42E0008ED2A00088B
:102F6000B02E0008852A000800F8010800127A0037
:042F7000000000005D
:04000005080000BD32
:00000001FF
